:020000040000FA
:08000000803102288731ED2F49
:100CC000FE0012001E00FE0B612E003406340534B7
:100CD000033402340134073408340434F200862E1D
:100CE000FC30AE2E6030AE2EDA30AE2EF230AE2EAC
:100CF0006630AE2EB630AE2EBE30AE2EE030AE2E0A
:100D0000FE30AE2EF630AE2E0030AE2E7208F00061
:100D1000F1017108003A03198E2E842E7008003AF2
:100D20000319702E013A0319722E033A0319742E17
:100D3000013A0319762E073A0319782E013A03195E
:100D40007A2E033A03197C2E013A03197E2E0F3AAC
:100D50000319802E013A0319822E842E0800F20016
:100D6000F301F601F7017208F0007608073C890AE2
:100D7000BA2EF036890BB92E701CBF2EC02ED12E84
:100D80000130F0007608203E860087010108FF3E12
:100D9000890ACB2EF035890BCA2E7008F100710834
:100DA000F3040130F6070030F73D7708803AF00091
:100DB00080307002031DDE2E08307602031CE12E07
:100DC000E22EB32E0730F4000030F5007308F00077
:100DD000740AEB2EF036890BEA2E7018F02EF32EE3
:100DE00020008E15F52E20008E110E160E12FF30EB
:100DF000F407FF30F53DF51FFE2EFF2EE62E8E1177
:100E00000800F601F31F052F062F0D2FF209F30935
:100E1000F20A0319F30AF601F60AF11F102F112F37
:100E2000162FF009F109F00A0319F10A700871048C
:100E300003191B2F1C2F452FF501F50A282F013010
:100E4000F035F10D890B202F0130F4007408F507FF
:100E5000F11F2B2F2C2F1F2F71087302031D322F10
:100E600070087202031C352F362F3A2F7008F202D9
:100E70007108F33B0130F136F00C890B3B2F013048
:100E8000F502031D442F452F2C2F76080319492FF7
:100E90004A2F4F2FF209F309F20A0319F30A7308D4
:100EA000F1007208F00008002100191599111916B7
:100EB00099161E169E121E179E130C1623000C1652
:100EC00021001D159D151D129D121D131D140E11BF
:100ED0008E110E128E1223000E118E11FF30200083
:100EE0009B0004309C002C009317131721009D14C5
:100EF0009D187B2F7C2F782F1C08F8007808FB00AA
:100F00007B082C0092000A30F0000030F1007C08D1
:100F10000B3EF200003003180130F3008731012747
:100F20008731700886316E2687318631AF2687314A
:100F30000A30F0000030F1007C08063EF20000307C
:100F400003180130F300873101278731700886319B
:100F50006E2687318631AF2687310A30F0000030A7
:100F6000F1007C08043EF200003003180130F30069
:100F7000873101278731700886316E2687318631A7
:100F8000AF2687317C0886316E2687318631AF26C1
:100F9000873120000E150E110130F9070030FA3D9F
:100FA0007A08803AF80080307802031DD92F643027
:100FB0007902031CDC2FDD2F762FF901FA010130B5
:100FC000F8007808FC070A307C02031CE82FE92FA0
:100FD000762FFC01762F803102286630840086301F
:100FE000850020308600003087000830863160267A
:100FF0008731F901FA01FB01FC0120008731542FF0
:020000040001F9
:04000E00A4C9CFDFD3
:00000001FF
